:020000040000FA
:0400000060283C3008
:08000800A000030EA100831209
:100010008B1C2E288B1031181328B11C2E2864300D
:100020000102031C2D281428152816281728182823
:1000300019281A281B283110B114A810031005190B
:100040000314AA0DA90DA80DB00B2E2831152A08EE
:10005000AF002908AE002808AD00B11081010B11D6
:0A006000210E8300A00E200E0900FF
:1000C000203084008001840A80300402031C6228EE
:1000D0001230B000272283160C3085058701831269
:1000E000850187010730990000309A00103083168F
:1000F0008E008312603083168F00831200308316C7
:1001000091009F008312C830831681008312313022
:100110009000003083168C00831210308B009822E0
:1001200081018E018F010B118B100B108C018B172D
:10013000B3203119C920F921B30BA6280310851962
:100140000314BA0DF0303A02031957210C1C9828F9
:100150000C10C00B98284108C00085013F30831661
:100160008500831298286400311808000B1D0800D0
:100170000B11B11031141230B000051DC428321417
:10018000831601138312080032108316011783129D
:100190000800321CD0282D090339AD00AE09AF0983
:1001A000E4302F02F0300319AF004C302F020C3036
:1001B0000319AF006C302F023C300319AF00EC3054
:1001C0002F02FC300319AF00B3302F02F3300319B4
:1001D000AF001B302F020F300319AF003B302F024E
:1001E0003F300319AF00BB302F02FF300319AF00BF
:1001F00031110130B7008B132030370783169B0075
:100200001C141A088312A400A5002510103037070B
:1002100083169B001C141A088312A30000303707B2
:1002200083169B001C141A088312A2008B17220845
:100230002D02031D512923082E06FC39031D5129C7
:10024000AF13AF12AF11AF1024082F02031D3A29CC
:1002500001303702031D31293E1831293E14B117F0
:100260004A2202303702031D3A29BE183A29BE1429
:10027000B117562225082F02031D512901303702DC
:10028000031D47293E1C47293E10B1176222023048
:100290003702031D5029BE1C5029BE10B1176E2213
:1002A0005129B70A0330370203180800FB28B601AA
:1002B000B301FA30B4000130B5000130B700850158
:1002C0008701B113D3218A22B320B30B8A290310EB
:1002D00085190314BA0DF0303A020319C229B41F6C
:1002E0008501B41F8701B40B8A29B50B8A29023016
:1002F000B50001303702031980220230370203199A
:1003000085223708B6080319B60003198829B603F1
:10031000FA30B400311D64293111321C94292D09A1
:100320000339AD00AE09AF0951302F065539031915
:10033000A92905302F0655390319A92915302F068B
:1003400055390319A92955302F0655390319A929FB
:100350006429AF13AF12AF11AF108B1320303707E2
:10036000BC002F08BB00072210303707BC002E0846
:10037000BB00072200303707BC002D08BB00072256
:100380008B17CD21912285018701B70AB601033071
:100390003702031C6429982208000230370203192F
:1003A0000800850187016430B900B320311DD529CB
:1003B0003111321CE0292D090339AD00AE09AF0916
:1003C00051302F0655390319D32905302F065539D9
:1003D0000319D32915302F0655390319D329553060
:1003E0002F0655390319D329B90BD5298501870162
:1003F0000800B11F0800B1131030BC003E08BB005C
:1004000007223030BC003F08BB00072208003C0830
:100410008B1383169B001C141A0883128B173B0244
:10042000031908008B133B0883161C159A008312CE
:100430003C0883169B0055309D00AA309D009C14FB
:1004400064009C18202A1C1183128B170800831645
:1004500000309B001C141A088312BD008316103054
:100460009B001C141A088312BE00831620309B00C8
:100470001C141A088312C1000130C11BC100C1083D
:100480000319C100831630309B001C141A08831214
:10049000BF0008008316051085108312051085140F
:1004A0008E018F010C104108C00008008316051250
:1004B00085128312051285168E018F010C104108DA
:1004C000C0000800831605108510831285100514DE
:1004D0008E018F010C104108C00008008316051220
:1004E00085128312851205168E018F010C104108AA
:1004F000C000080085013F30831685008312080084
:10050000380903398500B8000800380930398500FA
:10051000B80008003C30831685008312B801B81477
:1005200008000F30831685008312B801B816080042
:020530000800C1
:084000000800000006000200A8
:02400E00CC33B1
:10420000010003000300030003000200020002009B
:10421000020000000000FF00FF00FF00FF00FF00A1
:10422000000000000000000000000000000000008E
:104230000000C000C000FF00FF00FF00FF00FF0003
:104240000100510005001500550051000500150042
:10425000550051000500FF00FF00FF00FF00FF00B8
:104260000000FF00FF00FF00FF00FF00FF00FF0055
:10427000FF00FF00FF00FF00FF00FF00FF00FF0046
:10428000FF00FF00FF00FF00FF00FF00FF00FF0036
:10429000FF00FF00FF00FF00FF00FF00FF00FF0026
:1042A000FF00FF00FF00FF00FF00FF00FF00FF0016
:1042B000FF00FF00FF00FF00FF00FF00FF00FF0006
:1042C000FF00FF00FF00FF00FF00FF00FF00FF00F6
:1042D000FF00FF00FF00FF00FF00FF00FF00FF00E6
:1042E000FF00FF00FF00FF00FF00FF00FF00FF00D6
:1042F000FF00FF00FF00FF00FF00FF00FF00AA001B
:00000001FF
